:100000000C942A020C9462020C9462020C94620218
:100010000C9462020C9462020C9462020C946202D0
:100020000C9462020C9462020C94EC200C94282034
:100030000C9493250C9462020C9462020C9462025C
:100040000C9462020C94CA0F0C9462020C9462022B
:100050000C9462020C9452250C9462020C9462027D
:100060000C9462020C9462020C9462020C94620280
:100070000C9462020C9462020C9462020C94620270
:100080000C9462020C9462020C9462020C94620260
:100090000C9462020C9462020C9462020C94620250
:1000A0000C9462020C9462020C946202850785072C
:1000B000B707B70729084508DC09DC0950082E09ED
:1000C0003F093F09411E681E0020681E0020B01E27
:1000D000D31E0020C21FD51F000101010101010133
:1000E00001010202020202020202020303030303ED
:1000F00003030304040404040404050505050506BC
:100100000606060607070707070808080809090979
:10011000090A0A0A0B0B0B0C0C0C0D0D0D0E0E0E22
:100120000F0F0F10101111111212131314141515B3
:1001300016161717181819191A1A1B1B1C1D1D1E25
:100140001E1F202021222223242425262627282979
:10015000292A2B2C2D2D2E2F3031323233343536A7
:100160003738393A3B3C3D3E3F40414243444546A7
:100170004748494A4C4D4E4F505153545556585983
:100180005A5B5D5E5F616264656668696B6C6D6F2A
:100190007072737577787A7B7D7E8082838587889D
:1001A0008A8C8E8F91939596989A9C9EA0A2A3A5D7
:1001B000A7A9ABADAFB1B3B5B7BABCBEC0C2C4C6D8
:1001C000C9CBCDCFD1D4D6D8DBDDDFE2E4E7E9EB94
:1001D000EEF0F3F5F8FAFDFFFFAA7F554014001A80
:1001E000000800150029000400160007000900009F
:1001F0005CAA00A900BE00BD00000000047F3F1FF4
:10020000643214643214783C1E1E140A0505010978
:1002100002A10185020901A100050919012908159A
:100220000025019508750181020501093009311584
:1002300081257F95027508810609381581257F95EE
:100240000175088106050C0A38021581257F950184
:1002500075088106C0C005010980A1018503190147
:100260002AB700150126B700950175108100C00559
:100270000C0901A101850419012AA002150126A07B
:1002800002950175108100C005010906A10105074D
:1002900019E029E7150025019508750181029501EE
:1002A000750881010507190029FF150026FF009533
:1002B0000675088100050819012905950575019144
:1002C00002950175039101C009023B00020100A0E3
:1002D000FA090400000103010100092111010001D4
:1002E0002240000705810308000109040100010301
:1002F000000000092111010001227B000705820393
:10030000200001120100020000000812D8040001C0
:10031000000102000110034F00630074006F0070C1
:100320000061006400000026034E00650069006C57
:1003300000200042007200690061006E002000523F
:100340000061006D006900720065007A0000000421
:100350000309042223252628292A2C2D2F30323365
:100360003536383A3B3D3E4042434547494A4C4E7C
:100370005051535557595A5C5E6062646668696BA8
:100380006D6F71737577797B7D7F81838587898AAE
:100390008C8E90929496989A9C9E9FA1A3A5A7A8B4
:1003A000AAACAEAFB1B3B4B6B8B9BBBCBEBFC1C2E4
:1003B000C3C5C6C7C9CACBCCCDCED0D1D2D2D3D477
:1003C000D5D6D7D7D8D9D9DADADBDBDBDCDCDCDC95
:1003D000DCDDDDDDDDDCDCDCDCDCDBDBDBDADAD963
:1003E000D9D8D7D7D6D5D4D3D2D2D1D0CECDCCCBE5
:1003F000CAC9C7C6C5C3C2C1BFBEBCBBB9B8B6B403
:10040000B3B1AFAEACAAA8A7A5A3A19F9E9C9A9892
:10041000969492908E8C8A89878583817F7D7B7963
:10042000777573716F6D6B6968666462605E5C5A44
:100430005957555351504E4C4A4947454342403E07
:100440003D3B3A3836353332302F2D2C2A29282699
:100450002523220011241FBECFEFDAE0DEBFCDBF7F
:1004600004B603FE18C08091B9039091BA03A0911D
:10047000BB03B091BC038730904BA740B04B59F4FD
:100480001092B9031092BA031092BB031092BC03EE
:10049000E0E0F8E3099512E0A0E0B1E0EAEAFAE56D
:1004A00002C005900D92A638B107D9F723E0A6E85F
:1004B000B2E001C01D92A93BB207E1F70E942418E7
:1004C0000C94532D0C9400001F93CF93DF93CDB762
:1004D000DEB767970FB6F894DEBF0FBECDBF4B8B6C
:1004E0005C8B6D8B7E8B8F8B61111092F00286E09E
:1004F0009E01235F3F4FD901E82F1D92EA95E9F74E
:1005000095E0FE017396D90101900D929A95E1F75D
:100510009C894E895F897B897D879E876F87598BF0
:10052000488BF901DE01179601900D928A95E1F74B
:10053000CE0107960E94831681113EC086E0FE011F
:100540003796DE01119601900D928A95E1F7FF81B1
:10055000E8856A857B856115710531F0EF3F31F4DF
:1005600081E0FF3F19F403C081E001C080E080FD1D
:1005700023C02091B50230E0C90101968770992708
:100580004091E60250E08417950779F1F983EA83F8
:100590007D836C8396E0929FD001939FB00D1124D0
:1005A000AA54BD4FFE01319601900D929A95E1F744
:1005B0008093B5020E94F11516E08091E6029091B9
:1005C000B5028917F9F0189FC00111248A549D4F74
:1005D0000E9483168823B1F08091E60290E0019694
:1005E000877099278093E602E8CF0E940528109231
:1005F000B5021092E602EFEAF2E086E0DF011D921A
:100600008A95E9F767960FB6F894DEBF0FBECDBFA7
:10061000DF91CF911F9108958F929F92AF92BF92D9
:10062000CF92DF92EF92FF920F931F93CF93DF93BE
:10063000CDB7DEB72A970FB6F894DEBF0FBECDBF99
:10064000FC010081D18083819481892B39F01FEFD7
:10065000D11206C091E00F3F19F403C091E001C030
:1006600090E090FD9FC77F0185E0DE011696019026
:100670000D928A95E1F7F70122818E819F812223D5
:1006800049F00E94D926182F682F8E819F810E94E1
:100690005F2703C00E943227182F2FE0129FF0011E
:1006A000112435E0D39EE00DF11D1124E00FF11D62
:1006B000EE0FFF1FE352FE4F0591149100328CE5BF
:1006C000180779F4F7018281882309F488C26091C0
:1006D0003A0361FB992790F981E0892780FB61F952
:1006E0000CC00132FCE51F0779F4F70182818823F1
:1006F00009F475C260913A03626060933A0387E03F
:1007000090E00E942E2A6BC20232FCE51F0771F4B2
:10071000F70182818823F9F060913A036D7F60933D
:100720003A0387E090E00E942E2A15C005322CE59E
:10073000120709F032C2F7018281882361F080E05C
:1007400090E0ACEDB3E480931C0190931D01A09365
:100750001E01B0931F0180913A0380FF73C081FF97
:1007600071C0F7018281882309F46CC0C8018E51E1
:100770009C45029708F45DC660911C0170911D01B3
:1007800080911E0190911F019B01AC010E94C62A1D
:100790004B015C010E940A2ABC01990F880B990B3E
:1007A0000E94DA2B20E03EEF4FEF56E40E94372BF9
:1007B0002DEC3CEC4CE45DE30E948F2C20E030E01B
:1007C00040E85FE30E94C62AA50194010E948F2C95
:1007D00060930C0170930D0180930E0190930F01B3
:1007E0000E940A2ABC01990F880B990B0E94DA2BF0
:1007F00020E03EEF4FEF56E40E94372B2DEC3CEC0F
:100800004CE45DE30E948F2C20E030E040E85FE3A1
:100810000E94C62A20911C0130911D0140911E01A9
:1008200050911F010E948F2C609314017093150149
:10083000809316019093170163E070E084E091E0EB
:100840000E94B31C0D31FCE51F0741F4F7018281C2
:10085000882309F4F0C10E946629C6C20E31FCE566
:100860001F0741F4F7018281882309F4E4C10E9443
:100870004C29BAC20F31FCE51F0749F4F701828108
:100880008823D9F080913A0380FDF1CFE4CF0A327A
:10089000FCE51F0769F4F7018281882371F010924B
:1008A0003C0364E070E080E291E00E94B31C9CC2D3
:1008B0000B32FCE51F0779F3BEC1F7018281882363
:1008C00009F41EC21092A0030430FDE51F0758F47E
:1008D0000B3F2CE5120780F4C80182509C454497D9
:1008E00008F0F8C109C002363DE5130729F0063AC1
:1008F0008DE5180709F0EEC10E94F21490930203EF
:100900008093010301319CE5190709F4CEC008F07A
:1009100045C00930FCE51F0709F4A5C000F5053006
:100920003CE5130709F48DC078F403309CE5190702
:1009300009F47FC008F081C002301C4509F01DC1D8
:1009400080910103816017C107302CE5120709F47B
:1009500082C008F084C08091010380610CC10D3019
:100960008CE5180709F48DC070F40B30ECE51E0718
:1009700009F47FC008F081C0809101038860846021
:1009800080930103B3C00F302CE5120709F485C032
:1009900008F087C080910103877FEDC00E3F8CE592
:1009A000180709F476C008F50531ECE51E0709F4CF
:1009B0008EC068F403312CE5120709F47AC008F000
:1009C000B8C00E940528809101038F77D4C00C3FE6
:1009D0008CE51807D1F108F058C00B3F1C4509F011
:1009E000CCC080910203816033C00230FDE51F0757
:1009F00009F4ABC070F401153DE5130709F460C0BC
:100A000008F07EC0809102038260816080930203BF
:100A100084C002369DE5190709F49DC0063AEDE54C
:100A20001E0709F4A2C003301D4509F0A6C060E00E
:100A30008DC08091010382609EC08091010384601B
:100A40009AC080910103886096C080910203826001
:100A50008093020392C08091010380628CC08091D8
:100A60000103806488C00E9405288091010380688A
:100A700082C0809101038E7F7EC0809101038D7FB3
:100A80007AC0809101038B7F76C0809102038E7FB4
:100A9000DFCF809102038D7FDBCF809101038F7EBA
:100AA0006AC0809101038F7D66C0809101038F7BB6
:100AB00062C080910103877F8B7F809301031BC0FD
:100AC000809102038D7F8E7F809302032BC08091E3
:100AD000010382FB222720F991E0922790FB82F903
:100AE00090FB83F980930103992329F064E070E07F
:100AF00080E891E01BC062E070E080E591E016C004
:100B000080910203982F909591708E7F892B90FB96
:100B100081F980930203992329F064E070E080E674
:100B200091E004C062E070E080E491E00E94B31CB8
:100B300024C00E9405288091010387FB222720F909
:100B400091E0922790FB87F916C061E08EE090E07B
:100B50000E942E2A12C08091010384FB222720F9D3
:100B600091E0922790FB84F906C080910103982FB1
:100B7000909590FB80F9809301036091010310919F
:100B8000020384E090E00E942E2A612F82E290E02E
:100B90000E942E2A0E94052827C103323CE5130734
:100BA000F1F4F7018281882309F4D5CD29E038E3F7
:100BB00048E95FE360911C0170911D0180911E0165
:100BC00090911F010E948F2C4B015C0120E030E8C6
:100BD0004BEB54E40E94322B87FFBDCD23C004327F
:100BE0008CE5180709F0B7CDF7018281882309F455
:100BF000B2CD29E038E348E95FE360911C017091D0
:100C00001D0180911E0190911F010E94372B4B0105
:100C10005C0120E030E042E852E40E948A2C181681
:100C20000CF099CD80921C0190921D01A0921E01A2
:100C3000B0921F0190CD043F9CE5190749F406E2EC
:100C400021EE40EE64EF7CE5C7010E941B26CCC07C
:100C5000053FECE51E07F8F4093DFCE51F0731F4FC
:100C600007E225EE45EE69ED7CE5EECF0A3D2CE589
:100C7000120731F408E221E045EE6AED7CE5E4CFAD
:100C8000083D3CE5130709F018CE06E221EE41EEDF
:100C900068ED7CE5D9CF063F8CE5180731F406E214
:100CA00021EE42EE66EF7CE5CFCF063F9CE51907CB
:100CB00030F407E225EE44EE65EF7CE5C5CF073F53
:100CC000ECE51E0709F0F9CD07E225EE46EE67EFE9
:100CD0007CE5BACF0631FCE51F0721F58091F102D2
:100CE0008A7A91E009F490E090938802882311F0C9
:100CF00065E301C069E287EA92E00E94C9250FC05E
:100D000006312CE5120709F050C080918802882333
:100D100009F494C365E387EA92E00E94BC250E942F
:100D20007B1562C00B353DE51307C9F158F4011579
:100D30009CE51907B9F00F3D1C4509F08AC00E94D7
:100D4000031552C00C35FDE51F0759F10D351D4542
:100D500009F07FC08091020382FB882780F991E02F
:100D6000892720C00E9405280E9487258C0163E006
:100D700070E080EA91E00E94B31CC8010E947825CF
:100D80008A3F910538F48FE99FE00197F1F700C0A1
:100D90000000F3CF0E9425290E942E2525C081E066
:100DA00001C080E00E94D41554C08091F10282728B
:100DB0000D3C2CE5120709F4D5C3C8F1023D2CE522
:100DC000120709F4DFC308F46BC3053D2CE51207D5
:100DD00009F4DEC308F477C3063DECE51E0709F409
:100DE000DCC30E351D45A9F58091E702877009F433
:100DF000D9C3F7018281882309F4D4C38091020307
:100E000082FDD0C382E02A960FB6F894DEBF0FBEF3
:100E1000CDBFDF91CF911F910F91FF90EF90DF90A9
:100E2000CF90BF90AF909F908F900C94B715073CD8
:100E30009CE5190709F482C308F010C3043CFCE5E3
:100E40001F0709F471C308F0FBC2033C1C4509F4F9
:100E500046C3F70182810081D180882359F0802F19
:100E60009D2D0E94D926182F682F802F9D2D0E941E
:100E70005F2705C0802F9D2D0E943227182F2FE05D
:100E8000129FF001112435E0D39EE00DF11D1124D5
:100E9000E00FF11DEE0FFF1FE352FE4F859194917D
:100EA0000E9458138C01982EF701D280A580A2943D
:100EB0003FE0A3228091E7028770B9F0DD20A9F01E
:100EC000812F807F803421F080E2800F883068F0AD
:100ED0008091020382FD09C082E00E94B7158091D3
:100EE000E7028770CC24C3948111C12CB12EB29437
:100EF0009FE0B9228B2D90E08C30910508F05CC208
:100F0000FC01EA5AFF4F0C94242D812F807F1F7023
:100F1000882311F01295107FDD20B9F0112309F418
:100F200038C280E2800F883010F0911006C08091A6
:100F3000F102182B1093F10205C08091F002182BDA
:100F40001093F0020E947B1524C2802F0E9421285A
:100F5000112309F431C2005E083078F1992069F15B
:100F600010958091F00218231093F00229C0812F70
:100F7000807F1F70803211F01295107F992021F030
:100F8000F1E09F16D9F149C08091020382FF1BC096
:100F9000DD2069F0112339F08091F102182B1093B4
:100FA000F1020E947B1580E00E94812805C280E04A
:100FB0000E942128112309F4FFC1812F0E9474157A
:100FC0000E947B15F9C1DD2081F08091F202AA20F8
:100FD00051F001E0A01207C0182B181709F4ECC15A
:100FE0001093F202E9C1812B10C0AA2021F021E068
:100FF000A21609F4E1C10E946E1527C0DD2041F060
:1010000035E03A1508F4D8C1812F0E941728D4C1C1
:1010100084E08A1508F4D0C118C0DD2049F0AA2068
:1010200099F3F701858180FFB4C18F708583ECCF80
:10103000AA2059F0093309F0BCC1FFEF17EE23E0F5
:10104000F15010402040E1F7B2C1812F0E941028DA
:10105000B3C1812F86958695837019F0813059F040
:10106000ABC1DD2019F0C801937002C080E090E0B0
:101070000E94F925A7C1DD2019F0C801937002C0B4
:1010800080E090E00E94E3259DC1802FDD2019F0D3
:101090000E94940E02C00E94DB0D0E94B10D92C10D
:1010A000812F837009F069C0D1108AC1902F929569
:1010B00096959770990F990F802F8F70882E912C8D
:1010C000A12CB12C092E04C0880C991CAA1CBB1C95
:1010D0000A94D2F704FF12C04FE050E060E070E0E5
:1010E00004C0440F551F661F771F9A95D2F7DB0186
:1010F000CA0180959095A095B09503C080E090E0DE
:10110000DC0116951695412F4370423019F1C8F451
:101110000091F3021091F4022091F5023091F60251
:10112000413059F088299929AA29BB29BC01CD0150
:1011300060237123822393230AC0802A912AA22A42
:10114000B32ABC01CD01682979298A299B290E94EB
:10115000DB2736C188299929AA29BB290091F302E6
:101160001091F4022091F5023091F602BC01CD01FC
:101170006027712782279327EACFDD2019F0812F7E
:10118000817001C08695882309F41AC1902F929529
:1011900096959770990F990F802F8F70882E912CAC
:1011A000A12CB12C092E04C0880C991CAA1CBB1CB4
:1011B0000A94D2F704FF12C04FE050E060E070E004
:1011C00004C0440F551F661F771F9A95D2F7DB01A5
:1011D000CA0180959095A095B09503C080E090E0FD
:1011E000DC0116951695412F43704230D9F068F511
:1011F0000091FD021091FE022091FF023091000348
:10120000413059F088299929AA29BB29BC01CD016F
:1012100060237123822393231EC0802A912AA22A4D
:10122000B32A13C088299929AA29BB290091FD0254
:101230001091FE022091FF0230910003BC01CD010C
:10124000602771278227932706C0BC01CD0168293A
:1012500079298A299B290E948B27B2C01F70DD2023
:1012600039F0812F0E94BA27802F0E941728A8C02A
:10127000802F0E941028812F0E949527A1C0802FC7
:1012800032EF931609F443C0391538F090EF9916F0
:1012900059F0E1EF9E16B1F177C0F3EF9F16F1F12F
:1012A00024EF921659F170C0DD2019F134E03A159F
:1012B00008F482C01F7181E090E0A0E0B0E0AC01D2
:1012C000BD0104C0440F551F661F771F1A95D2F742
:1012D0008091FD029091FE02A091FF02B091000367
:1012E0008A019B01082719272A273B27C901B80132
:1012F00029C025E02A1508F45FC0DCCF80910203E5
:1013000082FF23C0DD2029F0812F8F7130C0DD20C6
:10131000D9F3812F8F710E9495274EC0DD2079F07F
:101320001F7181E090E0A0E0B0E0BC01CD0104C0FD
:10133000660F771F881F991F1A95D2F703C060E0C8
:1013400070E0CB010E948B2737C0DD2099F01F7120
:10135000812F0E94BA278091020382FD07C038E0E6
:10136000139FC001112483608093E702812F0E94A4
:10137000BA2722C081E00E94B71581E08A15E0F407
:1013800082E00E94B71518C0DD2029F0AA2009F4D8
:10139000BBCF802F09CEAA2009F4BBCF893349F4F3
:1013A0009FEFE7EEF3E09150E040F040E1F700C03E
:1013B0000000802F0E94212888EF8B0D843010F4CC
:1013C0000E940F26CC20A9F08091E70280FD11C079
:1013D000F70112828595859585950E94BA27C701E8
:1013E0000E940C038091E7028595859585950E9462
:1013F000952785E0F701DE01119601900D928A95FF
:10140000E1F789819A810E9432279A810FE0809FBB
:10141000F001112415E0919FE00DF11D1124898147
:10142000E80FF11DEE0FFF1FE352FE4F85919491DF
:10143000B9C00E311C4509F025CA19CA69E26BCC46
:10144000053C9CE5190709F474C0063C1C4509F0ED
:1014500000CD4AE45DE063E57DE088C00A3CFCE540
:101460001F0709F475C070F4083C3CE5130709F444
:101470006AC0093C1C4509F0ECCC4EE35DE062E338
:101480007DE074C00B3CECE51E0709F466C00C3C23
:101490001C4509F0DECC42EA5BE063EB7BE066C012
:1014A0000F3C8CE5180709F467C008F462C0003DE2
:1014B000ECE51E0709F463C0013D1C4509F0C9CCE9
:1014C0006EE089E067C0033D8CE5180709F45DC054
:1014D000043D1C4509F0BDCC61E088E160C080910D
:1014E000990380FF1BC08E7F8093990360919903BD
:1014F00070919A0380919B0390919C030E94900BA2
:101500001092A6020FEF10E722E001501040204099
:10151000E1F700C000000E94360B66CC816080932A
:10152000990361E086953BC04EE95DE067EA7DE0A6
:101530001DC047EA5DE06EE97DE018C043E55DE06F
:101540006AE47DE013C042E35DE06EE37DE00EC03F
:101550004AE15DE066E27DE009C046E25DE06AE105
:101560007DE004C043EB5BE062EA7BE00E94B826CA
:101570003BCC61E081E013C065E082E00BC068E035
:1015800086E008C064E18FE005C067E185E102C044
:1015900062E289E10E94A62627CC61E083E20E94F4
:1015A0005C0D22CC2A960FB6F894DEBF0FBECDBFDD
:1015B000DF91CF911F910F91FF90EF90DF90CF902F
:1015C000BF90AF909F908F900895CF92DF92EF924F
:1015D000FF926B017C0120E030E0A9010E94322BD8
:1015E000811106C0809180008F738093800039C084
:1015F00080918000806880938000C0928A02D0929F
:101600008B02E0928C02F0928D0220E030E040E00C
:1016100051E4C701B6010E948F2C9B01AC0160E030
:1016200074E284E79BE40E94372B6B017C010E94EB
:10163000A92B709387006093860020E030E048E497
:1016400052E4C701B6010E948F2C20E030E048EC44
:1016500052E40E94372B0E94A92B7093890060935B
:101660008800FF90EF90DF90CF90089580919903CC
:1016700080FF0AC0879A81B38F7791B390682FB7A4
:10168000F894E1E8F3E00BC0E1E8F3E011821082A6
:101690001282339633E0E939F307C1F7EBCF33E039
:1016A000E939F30789F0319148E091BB000000C0AF
:1016B00037FF81BB330F000000C000C000C081BBFA
:1016C00000C04A9591F7EBCF2FBF8FE594E00197CB
:1016D000F1F700C0000008959091990390FF0CC0AD
:1016E000E1E8F3E0818360834283339693E0E93954
:1016F000F907C1F70C94360B089580919903282FB0
:10170000269530E02115310519F48170826005C0FD
:101710002532310524F081708864809399030895FF
:10172000CF92DF92EF92FF926B017C010E947D0BC2
:10173000B701A60188E090E0FF90EF90DF90CF9096
:101740000C94402A80919D03882319F08150809346
:101750009D036091990370919A0380919B039091EE
:101760009C030C94900B80919D03833018F48F5F41
:1017700080939D036091990370919A0380919B03DC
:1017800090919C030C94900BE9E9F3E083E0808353
:1017900011828FEF828383831482608171818281C1
:1017A00093810C94900BAF92BF92CF92DF92EF9205
:1017B000FF920F931F93CF93DF93E82EF62EE9014C
:1017C000E42FF0E0611106C0E852FF4FE4914E2F84
:1017D0002E2F71C0062F10E0E852FF4F4491F42FD6
:1017E000C42ED12C26E0829FC00111242FEF30E0BF
:1017F000B9010E94FC2C5BEA5603C001579F900D73
:1018000011248E0D911D8E0D911D582F550F580FBF
:10181000D901A01BB10BAC9DC001AD9D900DBC9D2D
:10182000900D1124E92FF59ED0011124AB2FBB2779
:101830007901EA1AFB0AEC9CD001ED9CB00DFC9CEE
:10184000B00D11245901A51AB108A09E7001A19EE6
:10185000F00CB09EF00C1124EF2CFF242E193F0940
:101860002C9D80012D9D100D3C9D100D1124212FCC
:101870006230710591F048F461157105E1F0613055
:101880007105B9F4242F4B2F16C06430710569F02F
:1018900040F06630710579F00CC0242F492FE12FFC
:1018A0000AC0492FEF2F2B2F06C0292FE42F412FDD
:1018B00002C0292FEB2F49832883EA83DF91CF9140
:1018C0001F910F91FF90EF90DF90CF90BF90AF905E
:1018D0000895CF93DF9300D01F92CDB7DEB79091DC
:1018E000990390FF0AC09E012F5F3F4F0E94D30BC8
:1018F0004B8169818A810E946C0B0F900F900F9031
:10190000DF91CF9108957F928F929F92AF92BF9275
:10191000CF92DF92EF92FF920F931F93CF93DF93BB
:1019200000D01F92CDB7DEB7182FD62E042FC22EAF
:101930009091990390FF6DC0E92FE695AE2FB0E02E
:10194000A45FBD4F8C918093A5029E7F923061F47D
:101950009E012F5F3F4F812F0E94D30B4B816981E6
:101960008A810E946C0B43C0823019F400919C0361
:101970003EC0863019F410919A0339C08930D9F3EA
:101980008931A9F5E9512E2F2170722EE695F0E0EC
:10199000E852FE4F8590949031E8A32E33E0B32EA9
:1019A000E12CF12C99248E9CC0018F9C900D9E9C63
:1019B000900D112423E0969587952A95E1F77110F3
:1019C00002C0810F03C0212F281B822F9501402FB9
:1019D0006D2D0E94D30B8FEFE81AF80A23E0A20EB8
:1019E000B11C88E0E816F104F1F60E94360B109362
:1019F0009A03D0929B0300939C03CC2051F06091FA
:101A0000990370919A0380919B0390919C030E948B
:101A1000900B0F900F900F90DF91CF911F910F912E
:101A2000FF90EF90DF90CF90BF90AF909F908F90FE
:101A30007F900895E9E9F3E0438121E1421B08F436
:101A400040E021E0628181810C94830CE9E9F3E0BC
:101A5000438121E1420F08F44FEF21E0628181814F
:101A60000C94830CE9E9F3E0628121E1621B08F444
:101A700060E021E0438181810C94830CE9E9F3E08B
:101A8000628121E1620F08F46FEF21E043818181DF
:101A90000C94830CE9E9F3E0818121E043816281C8
:101AA00088500C94830CE9E9F3E0818121E04381C3
:101AB0006281885F0C94830C9091990390FF3DC0E4
:101AC0009170811102C0926006C0853210F0986456
:101AD00002C0880F982B90939903662351F0609170
:101AE000990370919A0380919B0390919C030E94AB
:101AF000900B60919903669570E04BE050E089EBA4
:101B000091E00E94392D892B19F01092A60209C08C
:101B100081E08093A6020E9487259093A002809383
:101B20009F0281E08093A20220E040919C0360919B
:101B30009B0380919A030C94830C089580919903E0
:101B40008695815009F484E261E00C945C0D8091EB
:101B5000990386958F5F853208F081E061E00C94EF
:101B60005C0D0E94872520919B02211104C02091C9
:101B70009C02222321F09093980280939702209157
:101B80009D02211104C020919E02222321F09093F6
:101B9000960280939502E091A303F091A4033097FD
:101BA00049F082E0809399020480F581E02D89E973
:101BB00092E0099408958D3E39F490919C0297FF2C
:101BC00035C010929C0259C08E3E29F490919C021F
:101BD0001916BCF32BC090919B028F3E29F497FFFE
:101BE00025C010929B0249C0803F19F41916CCF30E
:101BF0001DC090919D02893F29F41916BCF41092E2
:101C00009D023BC08A3F19F497FF10C0F8CF8B3F6D
:101C100039F490919E0297FF09C010929E022DC048
:101C20008C3F21F490919E021916BCF39FE0980F0F
:101C3000983080F421E030E0A90102C0440F551F24
:101C40009A95E2F7CA01809590919A028923809330
:101C50009A0213C08D3F21F4809194028E7F0BC0B5
:101C60008E3F21F4809194028D7F05C08F3F29F42F
:101C7000809194028B7F8093940280919B028111CA
:101C800006C080919C02811102C010929302809143
:101C90009D02811106C080919E02811102C01092A6
:101CA000920208958091940280FD16C081FD16C0B5
:101CB00082FD18C080919202882391F0883290F4BE
:101CC00028E0829FC001112468E270E00E94102D7C
:101CD000862F672B29F007C082E0089584E00895DD
:101CE00081E0089588E008958091940280FD14C0F9
:101CF00081FD14C082FD16C080919302882381F07B
:101D00008E3180F420E5829FC00111246EE170E0E5
:101D10000E94102D862F089584E1089588E2089589
:101D200088E0089580E508958D3E21F40E94740EA8
:101D3000819504C08E3E29F40E94740E80939C020B
:101D400008958F3E21F40E94740E819504C0803F57
:101D500029F40E94740E80939B020895893F19F420
:101D60000E94520E05C08A3F31F40E94520E8195A6
:101D700080939D0208958B3F21F40E94520E81951D
:101D800004C08C3F29F40E94520E80939E02089555
:101D90009FE0980F983078F421E030E0A90102C06C
:101DA000440F551F9A95E2F7CA0190919A02892B28
:101DB00080939A0208958D3F21F48091940281606E
:101DC0000BC08E3F21F480919402826005C08F3F4A
:101DD00029F4809194028460809394020895EFE640
:101DE000F0E080818D7F8083E0E8F0E080818F7378
:101DF000808308957F928F929F92AF92BF92CF92ED
:101E0000DF92EF92FF920F931F93CF93DF934B01DB
:101E10005C016A0180913A0380FFAEC08091390372
:101E2000811102C00E94752920E030E0A901C5019E
:101E3000B4010E94322B87FF04C0B7FAB094B7F800
:101E4000B09470907D03072D10E0E801219743E0E6
:101E5000000F111F4A95E1F7E12CF12CCF3FFFEF66
:101E6000DF07D9F128E0E21AF108F801EE0DFF1DB5
:101E7000E35CFC4F2281338144815581C501B4016B
:101E80000E94322B811127C08E0133E0000F111FF9
:101E90003A95E1F7035C1C4F80917D0390E0019738
:101EA000C817D9070CF068C0219688E0F801389669
:101EB000D80101900D928A95E1F70E948725F801DB
:101EC0009187808782869386A486B586D786C686C4
:101ED000085F1F4FE1CF2197C1CF81E0870D893087
:101EE00020F580937D0381E08093890280933803FD
:101EF000C0917D03D0E021970E948725FE0123E059
:101F0000EE0FFF1F2A95E1F7E35CFC4F918380837E
:101F100082829382A482B582D782C6820E9487255C
:101F20008091B801882341F113C088E080937D033C
:101F30008DE393E028E0FC013896DC0101900D92DE
:101F40002A95E1F7089623E08537920799F7CBCFDA
:101F500080916F00826080936F0080918000806824
:101F60008093800080913803882321F00E94861C92
:101F70000E94E50A1092B801DF91CF911F910F9155
:101F8000FF90EF90DF90CF90BF90AF909F908F9099
:101F90007F9008951F920F920FB60F9211242F92E7
:101FA0003F924F925F926F927F928F929F92AF92E9
:101FB000BF92CF92DF92EF92FF920F931F932F93D6
:101FC0003F934F935F936F937F938F939F93AF93C1
:101FD000BF93CF93DF93EF93FF9380918E02909105
:101FE0008F02A0919002B09191020196A11DB11DA6
:101FF00080938E0290938F02A0939002B0939102EF
:1020000060918E0270918F02809190029091910266
:102010000E94D82B6B017C0120E030E040E85CE3BB
:1020200060918A0270918B0280918C0290918D0256
:102030000E948F2C9B01AC01C701B6010E94322B7C
:1020400087FDBAC110928E0210928F0210929002F8
:102050001092910280913803811105C0C09137031D
:10206000CC2309F498C10E948725EC0180913703A5
:10207000811102C0312CE4C080912D0390912E0378
:102080000E94782520912B0330912C03821793070F
:1020900088F380912D0390912E030E947825209142
:1020A0002B0330912C037C01E21AF30AD0932E0308
:1020B000C0932D0300912F0310913003C8010196A6
:1020C0009093300380932F030E948725A0903203C2
:1020D000B090330380912F03909130038A159B05B4
:1020E00060F0C0913103CC2329F01092300310929C
:1020F0002F0303C00E9425294EC180913603C09151
:102100002F03D0913003C0903403D0903503811158
:1021100031C0F80163E0EE0FFF1F6A95E1F7EC0DA7
:10212000FD1DDE0173E0AA0FBB1F7A95E1F7AC0D30
:10213000BD1D2D913D914D915C9160817181828198
:1021400093810E94322B811115C081E08093360368
:102150004FE050E060E070E0CB010E94FA0E109377
:10216000300300932F038FE090E090932C03809333
:102170002B0364C0109236038E0143E0000F111F41
:102180004A95E1F70C0D1D1DF8016481758186816A
:1021900097810E94A92B9B01A0E6BAEE0E94B62A65
:1021A00020E03EE140E050E00E94942AF1E0AF1AC6
:1021B000B108412C5EE1552E612C712C2E153F0586
:1021C00050F0D0933003C0932F03E216F306E0F0F3
:1021D000C1E0D0E01CC0085F1F4FCA15DB0588F7BF
:1021E000E21AF30A2196F80164817581868197814C
:1021F0000E94A92B9B01A0E6BAEE0E94B62AA30179
:1022000092010E94942ADACFE901CE19DF09809168
:102210002F039091300333E0880F991F3A95E1F72F
:10222000F601E80FF91F6081718182819381AE010F
:102230000E94FA0ED0932C03C0932B0333243394C3
:1022400080913803882309F49EC080913B03882342
:1022500011F0332433940DE313E0812C912C412CA5
:10226000512C20E8622E2FEB722E22242394809191
:102270007D0390E0881699060CF085C0F8018681F0
:10228000978101978E3F9F4F08F077C0F8018081BA
:1022900091810E947825F801268137818217930762
:1022A00008F46BC0C280D380E480F58020E030E089
:1022B000A901C701B6010E94322B87FF04C0F7FABB
:1022C000F094F7F8F09480913803882309F455C00E
:1022D00080913903811102C00E9475299DE3A92EC6
:1022E00093E0B92EC7E0D0E0A7019601F50162ADF9
:1022F00073AD84AD95AD0E94322B811126C083E071
:10230000CC0FDD1F8A95E1F7C35CDC4F1982188280
:102310004A825B826C827D821F821E8285E793E007
:102320008C179D07D9F088E0FE013896DE010190F8
:102330000D928A95E1F7198618864A865B866C8627
:102340007D861F861E862896E9CF219798E0A91AD8
:10235000B108CF3FEFEFDE0739F60FC020928902B8
:1023600080917D03815080937D03811106C00E947E
:10237000EF0E2092B80110923803FFEF8F1A9F0AD8
:10238000085F1F4F74CFC0918902CC2319F01092BF
:10239000890201C0C32D80913803811107C080914B
:1023A0003703811103C00E94EF0E06C0CC2321F039
:1023B0000E94861C0E94E50AFF91EF91DF91CF9168
:1023C000BF91AF919F918F917F916F915F914F914D
:1023D0003F912F911F910F91FF90EF90DF90CF9041
:1023E000BF90AF909F908F907F906F905F904F9035
:1023F0003F902F900F900FBE0F901F90189580E088
:1024000008959091010392FF0DC0282F2871283064
:1024100019F4877F846006C0282F2471243011F4BA
:102420008B7F886093FF0DC0282F2871283119F405
:10243000877E846106C0282F2471243111F48B7E9D
:1024400088612091020320FF0DC0382F3871383089
:1024500019F4877F816006C0382F3171313011F453
:102460008E7F886021FF0DC0282F2871283119F434
:10247000877E816106C0282F2171213111F48E7E63
:10248000886194FD877E0895F894E82FE295EF70B7
:10249000F0E031A1282F2F7081E090E001C0880F7B
:1024A0002A95EAF7982F9095932391A392A1892BCF
:1024B00082A3789408955F926F927F928F929F92F9
:1024C000AF92BF92CF92DF92EF92FF920F931F9342
:1024D000CF93DF93CDB7DEB728970FB6F894DEBF62
:1024E0000FBECDBF1E821F82188602E612E07E015B
:1024F00046E0E40EF11C25E6C22E22E0D22E370182
:10250000AA24A394B12C4AE6842E42E0942EF8012A
:1025100080818F3F09F440C0F894E82FE295EF7076
:10252000F0E021A18F70A50102C0440F551F8A95CC
:10253000E2F7CA01922F982B91A392A1809589234B
:1025400082A3789400C0E5E6F2E0512C31E02191BD
:102550002F3F89F0A22FA295AF70B0E090968C919A
:1025600090E02F7002C0959587952A95E2F780FD3F
:1025700002C0832F01C080E0582A330F8E169F06B9
:1025800031F7F80180818F3F11F00E944412F0EA88
:10259000FA95F1F7F70150820F5F1F4FFFEFEF1A27
:1025A000FF0AC016D10609F0B2CF43E050E0B301F4
:1025B0008AEF92E00E94462DBB24B394009709F461
:1025C000B12C892B91F08E819F81A8858093FA028E
:1025D0009093FB02A093FC0281E08093F9020E9499
:1025E00087259093F8028093F7028091F90288235F
:1025F000B1F08091F7029091F8020E94782505973A
:1026000070F08091FA02809304038091FB02809322
:1026100005038091FC02809306031092F9020BE0FF
:1026200013E08EE6C82E82E0D82E9AE6E92E92E0DC
:10263000F92EF80180818823C1F0869511F0F6010A
:1026400001C0F701808191819A8389831B820E9456
:1026500087258160782F9D838C83F80110824981C2
:102660005A816B818D810E9464020F5F1F4FF2E0DF
:10267000CF0ED11C42E0E40EF11C53E00D301507E3
:10268000C1F68B2D28960FB6F894DEBF0FBECDBFD6
:10269000DF91CF911F910F91FF90EF90DF90CF903E
:1026A000BF90AF909F908F907F906F905F900895B4
:1026B000CF93DF938238910569F1B0F481339105AE
:1026C00009F46FC048F48932910509F465C08A3273
:1026D000910509F46BC08AC08533910509F457C090
:1026E00089339105B9F082C0833E910571F138F4C8
:1026F000803E9105B1F0823E910511F177C0863E92
:102700009105B9F1873E9105C9F1843E910509F023
:102710006DC024C02091010320FD53C021FD51C094
:1027200065C08091010380FD46C08091020380FF57
:1027300048C08091010384FD50C183EE90E04FC1F9
:102740008091010382FF3AC0F4CF8091010382FDA2
:1027500035C08091020380FD34C0EBCF809102032D
:1027600081FF35C08091010384FD37C187EE90E081
:1027700036C18091010383FF27C0F4CF809101030C
:1027800083FD22C08091020381FD21C0EBCF8091A7
:10279000010385FD1FC021C08091010385FD1DC07F
:1027A00019C08091010386FD1BC01DC080910103EB
:1027B00086FD19C015C089E390E011C182EE90E05A
:1027C0000EC180EE90E00BC186EE90E008C184EE71
:1027D00090E005C189E290E002C185E390E0FFC08E
:1027E0008AE290E0FCC081E390E0F9C0811531E518
:1027F000930708F069C0811540E59407F0F09C014B
:1028000074E0369527957A95E1F7922F9370482FCB
:10281000437021E030E002C0220F331F4A95E2F7F7
:102820003C68392B982F9F709695969540E2949F1F
:10283000C0011124822B932BD2C0883E910568F5EC
:10284000803E910508F0CBC0883A9105B8F4853AEE
:10285000910548F0855AE82FF0E0EF5CFD4F80814C
:1028600090E09064BCC08130910509F4B3C008F4D5
:10287000B4C08430910508F4B0C0B1C08F3B91055D
:1028800008F0ABC0885AE82FF0E0EE0FFF1FEC5CB9
:10289000FD4F808191819464A2C0811520E292074E
:1028A00058F4811531E0930708F099C08D3E9105E9
:1028B00008F493C0906593C0811540E4940708F430
:1028C0008CC09F70906A8BC0811525E5920708F037
:1028D00042C0811534E5930728F0982F8827846F2C
:1028E000906A7DC0811543E59407B0F09C01237088
:1028F000332741E050E002C0440F551F2A95E2F70C
:10290000282F2695269580E2289F90011124CA0140
:10291000822B932B9A6863C0811522E5920728F4D5
:10292000982F8827816F906A5AC09C0123703327A3
:1029300041E050E002C0440F551F2A95E2F7282FCE
:102940002695269580E2289F90011124CA01822BAA
:10295000932B9C6844C0EC01811539E59307A8F4DA
:102960008115984528F09C2F8827806F906A37C082
:10297000C11586E5D80788F58C2F0E9401128F714A
:1029800090E0982F882790622AC081152AE5920747
:1029900090F48C2F8F700E94011294E0D695C79509
:1029A0009A95E1F7CF70D0E0DC2FCC27D0699E015B
:1029B000282BC90114C090568115904270F48D2FB8
:1029C0008F710E940112282F2F71CE0199279062DA
:1029D000922B05C081E090E002C080E090E0DF91A2
:1029E000CF910895CF9384E090E00E941A2AC82FD7
:1029F00082E290E00E941A2A2C2F30E0A901582B85
:102A0000CA01CF91089569EE7EEF80E090E00E94C8
:102A10004C2A60E082E090E00E942E2A60E083E091
:102A200090E00E942E2A1092F3021092F40210926B
:102A3000F5021092F60260E084E090E00E942E2AF7
:102A400060E082E290E00E942E2A60E085E090E063
:102A50000E942E2A60E086E090E00E942E2A6FEF0E
:102A600087E090E00E942E2A40E050E0BA0188E022
:102A700090E00E94402A60E08DE090E00E942E2AC3
:102A800040E050E0BA0188E190E00E94402A60E016
:102A900087E190E00E942E2A40E050E0BA018CE1EC
:102AA00090E00E94402A60E070E080E290E00E94A6
:102AB0004C2A40E050E0BA0188E190E00E94402AB0
:102AC00040E050E0BA018FE090E00E94402A40E0F0
:102AD00050E0BA0183E190E00C94402A8091F20228
:102AE00081111092F202089580959091F10289234C
:102AF0008093F10208959091F1028091F002982B59
:102B00009093A7028091F202882389F0892B809309
:102B1000A702E9EAF2E097E080E0915029F02191E4
:102B20002223D9F38F5FF9CF81110E946E1548E0FF
:102B300050E068EE72E087EA92E00E94462D892B11
:102B4000A9F088E0E7EAF2E0A8EEB2E001900D9289
:102B50008A95E1F7E091A303F091A403309731F057
:102B60000280F381E02D87EA92E009940895209194
:102B7000E702809582238093E702982F977099F45B
:102B800030E0482F082E000C550B2417350759F05C
:102B90009091020392FD07C08595859585950E94C9
:102BA00095271092E7020895CF93C0910203C2FBCC
:102BB000992790F9981799F080FBC2F9C093020306
:102BC0006091010384E090E00E942E2A6C2F82E243
:102BD00090E00E942E2A82E0CF910C94B715CF91FD
:102BE00008958091E6029091B502891719F08F5FE0
:102BF0008770FBCF08950F931F93CF93DF9380913E
:102C0000B40282958F7009F05DC08091B102882373
:102C100009F458C08091E6021091B5026091AF02AC
:102C20007091B002C091B202D091B30291E06F3FB7
:102C300009F090E0292F06E0811709F443C020979E
:102C400021F07F3F21F030E003C031E001C0322F9E
:102C500090E030FD34C0089FF001099FF00D112471
:102C6000DF01AA54BD4F11963C911197371327C02D
:102C70003C91361324C012963C91129731111FC01B
:102C800013964D915C9114974C1B5D0B483C51057C
:102C9000B0F48091B4028F7080618093B402E554E7
:102CA000FD4F80818F70806180838FEA92E00E9467
:102CB0000C03DF91CF911F910F910C94F1150196A8
:102CC0008770BACFDF91CF911F910F910895CF9365
:102CD000DF93EC010E94D9262FE0829FC0011124CE
:102CE000FC0125E0D29FE00DF11D1124EC0FF11D38
:102CF000EE0FFF1FE352FE4F859194910E945813EF
:102D0000DF91CF9108959F92AF92BF92CF92DF92C1
:102D1000EF92FF920F931F93CF93DF93CDB7DEB760
:102D200061970FB6F894DEBF0FBECDBF8C0185E072
:102D3000F801DE011D9601900D928A95E1F7F801E8
:102D4000E2809091AF026091B0024091B202509146
:102D5000B3024115510531F06F3F31F481E09F3FDF
:102D600019F403C081E001C080E0F82FF1709F2EBC
:102D700080FD1AC1F80130812181C380D4808FEA9F
:102D8000A82E82E0B82EF090B102F601E41BF50BFC
:102D9000FF2009F4C6C08091B402E83CF10508F0B8
:102DA00091C0482F407F09F050C0621311C09313A7
:102DB0000FC0FE2CE1100CC08F7080618093B402B4
:102DC000C5010E940C038091B402F801858329C1DA
:102DD000CD2831F02F3F31F481E03F3F19F403C09B
:102DE00081E001C080E080FD03C081E08E2502C04B
:102DF00080E090E0F82FF170FF2E80FF1CC08091E2
:102E0000E6024091B50256E0841709F4E8C090E06C
:102E1000589FF001599FF00D1124EA54FD4F618134
:102E2000261306C06081631303C06281E61203C0EB
:102E300001968770E9CFFE2CEE2009F4F2C0809154
:102E4000B40281608093B40249C0621306C0931338
:102E500004C0E11002C0F80186C0C8010E94E52745
:102E6000882351F1EE2041F12091B402822F829506
:102E70008F7090E0029774F08091AF029091B00251
:102E800098878F831986DB86CA862C87CE010796A2
:102E90000E940C0386E0F801AFEAB2E001900D92C7
:102EA0008A95E1F70E94FB150AC06217C9F0C801B4
:102EB0000E94E52781111EC0C8010E940C03FF2457
:102EC000F394AFC0482F407F81F78FEA92E00E94D1
:102ED0000C0386E0F50111928A95E9F7F12CA1C067
:102EE0009313E5CFE110E3CFF8018583C8010E9479
:102EF0000C0354C0EE2001F32091B402822F82957E
:102F00008F7090E0029734F28091AF029091B002FE
:102F10009A8389831B82DD82CC822E83CE01019627
:102F2000B7CFE83CF105D0F5FE2CEE2029F2621374
:102F300027C0931325C02091B40220FD18C0822F12
:102F400082958F70482F50E04115510581F0F801AE
:102F500025834F30510541F08F5F982F9295907FD8
:102F6000822F8F70892B8583C8010E940C0386E015
:102F7000F801AFEAB2E001900D928A95E1F751C0F5
:102F8000C8010E94E527811185CF8091B40281603C
:102F90008093B402C8010E940C0343C086E0F5018F
:102FA00011928A95E9F73DC0EE2009F485CFC8015A
:102FB0000E94E527F82E882309F47ECF86E0F801E9
:102FC000AFEAB2E001900D928A95E1F78091AF02ED
:102FD0009091B0020E9467160E94FB1522C03D87A7
:102FE0002E878D859E850E946716292F22952F702A
:102FF000223028F49F7039F0811105C00BC02430B5
:1030000028F49F7049F4805E883020F0C8010E9447
:103010000C039F2CF92C05C0F8019581907F99F73E
:10302000F9CF8F2D61960FB6F894DEBF0FBECDBFDE
:10303000DF91CF911F910F91FF90EF90DF90CF9094
:10304000BF90AF909F900895CF93DF93CDB7DEB739
:1030500068970FB6F894DEBF0FBECDBF84B7877FE9
:1030600084BF0FB6F894A895809160008861809322
:103070006000109260000FBE90E080E80FB6F894F8
:1030800080936100909361000FBE85B7806885BF13
:1030900085B7806885BF8FEF91E190938702809319
:1030A00086020E946C200E948B208091E200846046
:1030B0008093E2007894809121038823A1F01091FD
:1030C000E9001F709091EC00892F817090FD80E8DD
:1030D000182B1092E9008091E80083FD0E945B1D8F
:1030E0001F701093E90082E084BD93E095BD9AEFD4
:1030F00097BD80936E0082E30E94441283E30E9496
:10310000441205E612E06AE6E62E62E0F62ED801E9
:103110008D918D018F3F11F00E944412E016F1064F
:10312000B1F783E0E4E0F3E0DF01E82E1D92EA94DA
:10313000E9F7EAEFF2E0DF011D928A95E9F780E016
:1031400090E00E94282A893E9E4F11F00E940315AC
:1031500082E090E00E941A2A809307030E94F214F2
:1031600090930203809301030E945B12EFE3FCE95A
:103170003197F1F700C000000E945B1280910403B8
:1031800080FF08C06FEF7FEF80E090E00E944C2A44
:103190000E942E2583E090E00E941A2A682F70E09A
:1031A00080E090E00E94DB270E9475298091030354
:1031B000811136C080E090E00E94282A893E9E4F0F
:1031C00021F00E9403150E94C40B88E090E00E9449
:1031D000222A6093990370939A0380939B039093A0
:1031E0009C036E7F71F40E94C40B88E090E00E9403
:1031F000222A6093990370939A0380939B03909380
:103200009C030E947D0B1092A6028091990380FF7F
:1032100004C060E086950E945C0D81E0809303030A
:1032200066E872E022E832E0A4E8B2E041E050E073
:103230006A177B0769F18D91E82FE295EF70F0E056
:1032400011A18F707A0102C0EE0CFF1C8A95E2F783
:10325000C7019E2D9095912391A392A1892B82A3C2
:10326000F90181919F01E82FE295EF70F0E011A143
:103270008F707A0102C0EE0CFF1C8A95E2F7C7013D
:103280009E2D9095912391A392A1892B82A3D0CFBB
:103290008FE891E00197F1F700C0000086B190E05F
:1032A000880F892F881F990B369902C020E001C032
:1032B00022E0822B809311038FB1829581707D99DA
:1032C00002C090E001C092E0892B8093120384EC4D
:1032D00091E09093A4038093A30338E1232E312C33
:1032E00040E4442E80912103853009F047C000E17D
:1032F00012E180912103853009F03CC080912103C7
:10330000843019F10E9425291092A7030FB6F89472
:10331000A895209260000FBE4092600083B7817F25
:10332000846083BF83B7816083BF7894889583B7B7
:103330008E7F83BF0FB6F894A89580916000886156
:1033400080936000109260000FBE8091200388235C
:1033500009F4CFCF0E945B12809104038111B6C2A1
:10336000809105038111B2C280910603882309F47C
:10337000C0CFACC20E9405280E940F260E945B129B
:10338000882359F08FB7F8944091A8035091A9036E
:103390006091AA037091AB038FBFE4E0F3E0A8E073
:1033A000B3E000E010E0302F21919D91922721F1B0
:1033B00080E0FF24F394492F4F21D1F08F83388789
:1033C0002F2181E009F480E089870E9487258160B0
:1033D000782F9B878A874F81588569858B850E94C6
:1033E0006402F801E85FFC4F8081F826F08219C082
:1033F0008F5FFF0C8530F9F60F5F1F4F033011050B
:1034000091F68FEF8C878D871E860E9487258160BD
:10341000782F988B8F874C855D856E8588890E9473
:1034200064028091A602882309F493C08091A502CA
:10343000E0919903E695E81BE093A102823059F4EC
:10344000F0E0E75FFD4FE4910E2F10E025E3E22E60
:1034500024E2F22E59C0863059F4F0E0EA5FFD4FC5
:10346000E4910E2F10E095E2E92E94E2F92E4CC083
:10347000893061F4E695F0E0ED5FFD4FE4910E2FA9
:1034800010E08BEBE82E83E2F82E3EC08F3061F423
:10349000E695F0E0E050FE4FE4910E2F10E0B7E526
:1034A000EB2EB3E2FB2E30C0853159F4F0E0E3504F
:1034B000FE4FE4910E2F10E0A9E0EA2EA3E2FA2ECF
:1034C00023C08831A1F0833249F4EBEFF1E005919C
:1034D0001491F5EEEF2EF3E2FF2E16C0843271F454
:1034E00004EF11E0E6E4EE2EE2E2FE2E0DC008E26B
:1034F00010E070E8E72E72E2F72E06C000ED17E04C
:1035000067ECE62E61E2F62E8091A202882361F03C
:103510001092A2020E9487259093A00280939F029E
:103520001092A4021092A3020E948725E0919F02AC
:10353000F091A0028E1B9F0B8F3F9F4750F40E0F00
:103540001F1F1093A00200939F028FE992E0F701E2
:10355000099521E133E03E8B2D8B8FE0E82E83E04F
:10356000F82E0DE013E09EE6892E92E0992E4BE0B6
:10357000C42E43E0D42E5AE6A52E52E0B52E82E8A2
:1035800092E09A8B898BA4E8B2E0BC8BAB8B388F2E
:103590002F8B712C612C55245394AF89B88D8D914C
:1035A000B88FAF8BE82FEE0FEE0FAB89BC892D9152
:1035B000BC8BAB8BA22FA295AF70B0E090968C9194
:1035C00090E02F7002C0959587952A95E2F79C01AF
:1035D00021703327A989BA898D91BA8BA98BA82F1D
:1035E000A295AF70B0E090964C9150E08F7002C001
:1035F000559547958A95E2F7CA018170992740FF52
:1036000002C082E090E0822B932B8E2BED89FE8905
:103610008193FE8BED8B8F70E82FF0E0EE58FD4F1D
:103620009081D7018C91890F8C938430D4F0F8016C
:1036300080818F5F8083D5018D919C919A8389834E
:103640005B820E9487258160782F9D838C83F601A1
:10365000508249815A816B818D810E94640221E0F0
:1036600001C020E0D7018C918D3FD4F4F801808116
:1036700081508083D4018D919C919A8389835B8250
:103680000E9487258160782F9D838C8322E0F6013C
:10369000208349815A816B818D810E94640221E0DF
:1036A000D7018C91082E000C990B64E070E00E9409
:1036B000102DF70181937F01722A63940F5F1F4FD2
:1036C000F2E08F0E911C2FEFC21AD20A32E0A30E45
:1036D000B11C42E0641261CF772059F08FB7F894A3
:1036E0004091A8035091A9036091AA037091AB0384
:1036F0008FBF86E0E9E9F2E0DE01119601900D92BC
:103700008A95E1F7E0909B02F0909C0200919D0267
:1037100010919E0210929B0210929C0210929D02A8
:1037200010929E02E11003C0FF2009F451C0809165
:103730009702909198020E9478259C0190919302A3
:10374000992309F4D9C02531310508F441C09F3FC0
:1037500019F09F5F90939302EE2061F00E94740E27
:103760001E1414F09FEF01C091E0899F802D112459
:1037700080939B02FF2061F00E94740E1F1414F0CE
:103780009FEF01C091E0899F802D112480939C02BE
:1037900030919B023323E1F020919C022223C1F05F
:1037A00045EB3403C0011124992319F090939B0237
:1037B00003C081E080939B0235EB2303C0011124F9
:1037C000992319F090939C0203C081E080939C029E
:1037D000011103C0112309F451C080919502909109
:1037E00096020E9478259C0190919202992309F4F7
:1037F00088C02135310508F441C09F3F19F09F5F13
:1038000090939202002361F00E94520E101614F061
:103810009FEF01C091E0899F802D112480939D022C
:10382000112361F00E94520E111614F09FEF01C097
:1038300091E0899F802D112480939E0230919D02FA
:103840003323E1F020919E022223C1F045EB3403A3
:10385000C0011124992319F090939D0203C081E0C7
:1038600080939D0235EB2303C0011124992319F0A5
:1038700090939E0203C081E080939E0280919B0200
:1038800081110BC080919C02811107C080919D0223
:10389000811103C080919E0281110E94B10DEB82C3
:1038A000FC820D831E8386E0FE013196A9E9B2E019
:1038B00001900D928A95E1F70E940F2690911303D3
:1038C000891709F40FCD809313030CCD09BD19BDE1
:1038D00009B400FEFDCF8091D8008F7D8093D80081
:1038E0008091E00082608093E0008091E00081FDA3
:1038F000FCCF0E940528FDCC2B30310508F029CFE4
:1039000067CF2B30310508F07ACFB8CFCF92DF9256
:10391000EF92FF92E0917D03EE23D9F0E15088E031
:10392000E802F0011124E35CFC4FC280D380E48004
:10393000F58020E030E0A901C701B6010E94322BDA
:1039400018163CF480913C03811106C010923B0391
:1039500003C0C12CD12C7601C701B601FF90EF90B6
:10396000DF90CF900895CF92DF92EF92FF92CF93A6
:10397000DF9320913A0320FD08C0DF91CF91FF90A3
:10398000EF90DF90CF900C9425297B01EC01809182
:103990003903811102C00E94752980913803811179
:1039A0000E94252981E08093370310923603D0933B
:1039B0003503C0933403F0923303E0923203109244
:1039C00031031092300310922F036C817D818E8120
:1039D0009F810E94A92B9B01A0E6BAEE0E94B62A05
:1039E000C12C2EE1D22EE12CF12CA70196010E94D0
:1039F000942A688179818A819B81A9010E94FA0EAB
:103A00000E94872590932E0380932D038091340389
:103A100090913503E0912F03F091300333E0EE0FE6
:103A2000FF1F3A95E1F7E80FF91F648175818681E0
:103A300097810E94A92B9B01A0E6BAEE0E94B62AAC
:103A4000A70196010E94942A30932C0320932B0304
:103A5000DF91CF91FF90EF90DF90CF900895EF929C
:103A6000FF920F931F93CF93DF937C018B010E94F2
:103A70004924811119C0E70101151105A1F08091B8
:103A8000E80085FD0AC08091E8008E778093E80009
:103A90000E944924882381F307C089918093F10013
:103AA00001501109E9CF80E0DF91CF911F910F9173
:103AB000FF90EF9008951F93CF93DF93CDB7DEB7BC
:103AC000AA970FB6F894DEBF0FBECDBFE3E2F3E0D6
:103AD0008BE293E02091F10021938E179F07D1F79D
:103AE00080912403833009F461C030F4813071F097
:103AF000823009F49BC0B2C08A3009F487C08B3091
:103B000009F46CC0893009F0A9C020C0809123035A
:103B1000813A09F0A3C08091E800877F8093E80094
:103B20008091270390912803892B21F468E087E195
:103B300093E003C060E080E090E070E00E94D02459
:103B40008091E8008B778093E80088C08091230300
:103B5000813209F083C08091270390912803029756
:103B600008F07CC08091E800877F8093E800809116
:103B7000E80082FD05C0809121038111F8CF6EC05D
:103B80002091F3008091F20090E0922B029731F4A3
:103B90008091F100813011F0863021F48091F100A4
:103BA000809316038091E8008B7754C080912303A3
:103BB000813A09F053C08091270390912803892B03
:103BC00009F04CC08091E800877F8093E8008091E5
:103BD000E80080FFFCCF8091D00137C080912303A3
:103BE0008132E1F58091270390912803892BB1F56B
:103BF0008091E800877F8093E8000E947C24809178
:103C000025038093D0010E94052828C080912303BA
:103C1000813221F58091E800877F8093E8000E943F
:103C20007C24809126038093150318C08091230380
:103C3000813AA1F48091E800877F8093E800809129
:103C4000E80080FFFCCF809115038093F100809104
:103C5000E8008E778093E8000E947C248091E80041
:103C600083FFCEC18091230390912403492F50E01C
:103C70004A30510508F0C4C1FA01EE59FF4F0C94C7
:103C8000242D803821F0823809F0BAC108C0809113
:103C90001F0390912003992389F082600FC08091C7
:103CA00027038F70873008F0ABC18093E9008091C3
:103CB000EB0085FB882780F91092E9009091E800DD
:103CC000977F9093E8008093F1001092F10065C116
:103CD000282F2D7F09F094C1882319F0823061F0DC
:103CE0008FC180912503813009F08AC1933009F09A
:103CF00080E0809320032EC08091250381112AC08B
:103D0000809127038F702FEF280F263008F078C19D
:103D10008093E9002091EB0020FF1CC0933021F438
:103D20008091EB00806214C09091EB0090619093C1
:103D3000EB0021E030E0A90102C0440F551F8A9535
:103D4000E2F74093EA001092EA008091EB0088606D
:103D50008093EB001092E9008091E800877F20C1FA
:103D600081114EC1109125031F778091E300807867
:103D7000812B8093E3008091E800877F8093E800A7
:103D80000E947C248091E80080FFFCCF8091E300BA
:103D900080688093E300111102C082E001C083E0DB
:103DA000809321032DC18058823008F029C1809171
:103DB0002503909126038C3D53E0950779F583E028
:103DC0008A838AE289834FB7F894DE01139620E054
:103DD0003EE051E2E32FF0E050935700E49120FFE2
:103DE00003C0E295EF703F5FEF708E2F90E0EA30F6
:103DF00010F0C79601C0C0968D939D932F5F24311C
:103E000049F74FBF8091E800877F8093E8006AE21E
:103E100070E0CE0101960E94D024AEC040912703ED
:103E200050912803292F332723303105A9F068F456
:103E30002130310509F4F3C02230310509F0E0C02A
:103E40008BE390E0E8ECF2E044C02132310521F14F
:103E50002232310571F1D4C0992781309105A1F04A
:103E600058F0029709F0CCC0E5E1F3E0E4918E2F21
:103E700090E0E5E1F3E02AC0EFE4F3E0E4918E2F77
:103E800090E0EFE4F3E022C0E7E2F3E0E4918E2F6C
:103E900090E0E7E2F3E01AC04115510509F4C4C00F
:103EA0004130510509F0ACC089E090E0E3EFF2E069
:103EB00010C04115510509F4BCC04130510509F04D
:103EC0009FC08BE790E0EDE0F2E003C0009709F4BB
:103ED00097C02091E800277F2093E80020912903D4
:103EE00030912A038217930708F49C0140E02115C2
:103EF000310589F180912103882309F43DC0853083
:103F0000D9F18091E80083FD37C08091E80082FDFF
:103F10002FC08091E80080FFEACF4091F3008091AC
:103F2000F20090E0942B2115310559F0883091056D
:103F300040F444914093F1003196215031090196AB
:103F4000F2CF41E0089709F040E08091E8008E77D9
:103F50008093E800CCCF4111CDCF0AC080912103DE
:103F6000882351F0853041F08091E80083FD04C042
:103F70008091E80082FFF2CF8091E8008B778093F8
:103F8000E8003EC08038E1F58091E800877F8093AB
:103F9000E800809122038093F1008091E8008E7701
:103FA0008093E8000E947C242BC0811129C080915D
:103FB0002503909126039927029714F58091E80034
:103FC000877F8093E80010912503109322030E94BD
:103FD0007C24111106C08091E30087FD02C081E0BE
:103FE00001C084E08093210342E061EC81E00E9403
:103FF0009B2442E261EC82E00E949B248091210399
:104000008091E80083FF1AC08091E800877F809349
:10401000E8008091EB0080628093EB000FC082E1AA
:1040200090E0E3E0F3E055CF89E090E0EAEDF2E0E4
:1040300050CF80E490E0E8E8F2E04BCFAA960FB6CC
:10404000F894DEBF0FBECDBFDF91CF911F910895D1
:104050001F920F920FB60F9211242F933F934F93FD
:104060005F936F937F938F939F93AF93BF93CF9300
:10407000DF93EF93FF93C091E900CF708091EC0044
:10408000D82FD17080FDD0E81092E9008091F00027
:10409000877F8093F00078940E945B1D1092E90066
:1040A0008091F00088608093F000CD2BCF70C0939A
:1040B000E900FF91EF91DF91CF91BF91AF919F9177
:1040C0008F917F916F915F914F913F912F910F90C1
:1040D0000FBE0F901F901895E8EDF0E080818E7F65
:1040E00080831092E2001092DA001092E100A0EEBC
:1040F000B0E08C9181608C9380818F77808319BC34
:10410000A7EDB0E08C918E7F8C9380818F7E808331
:10411000109214030895CF92DF92EF92FF920F93C3
:104120001F93CF93DF93C8EDD0E088818F7E888383
:10413000E7EDF0E080818160808384E082BF81E0F0
:104140008093140388818E7F888302EE10E0F8014B
:1041500010821092DA0081EEC82ED12CF601108266
:1041600088818F77888388818068888388818F7D24
:10417000888319BC1092210310922203109220030D
:1041800010921F0390EEE92EF12CF70180818B7FB6
:10419000808388818160888342E060E080E00E94C3
:1041A0009B24F60180818E7F8083F801808181606D
:1041B0008083808188608083F70180818E7F808307
:1041C000888180618883DF91CF911F910F91FF904B
:1041D000EF90DF90CF9008951F920F920FB60F923D
:1041E00011242F933F934F935F936F937F938F93FC
:1041F0009F93AF93BF93EF93FF938091E10082FF72
:1042000009C08091E20082FF05C08091E1008B7FB0
:104210008093E1008091DA0080FF2AC08091D8006D
:1042200080FF26C08091DA008E7F8093DA00809133
:10423000D90080FF18C080E189BD82E189BD09B441
:1042400000FEFDCF81E08093210380911403811152
:104250000FC00E946C200E948B208091E20084603D
:104260008093E20005C019BC109221031092140340
:104270008091E10080FF17C08091E20080FF13C0B1
:104280008091E2008E7F8093E2008091E200806165
:104290008093E2008091D80080628093D80019BC9E
:1042A00085E0809321038091E10084FF30C08091FC
:1042B000E20084FF2CC080E189BD82E189BD09B4A0
:1042C00000FEFDCF8091D8008F7D8093D800809133
:1042D000E1008F7E8093E1008091E2008F7E8093E9
:1042E000E2008091E20081608093E20080912203ED
:1042F000882311F084E007C08091E30087FD02C0AD
:1043000081E001C083E080932103809121038091AB
:10431000E10083FF27C08091E20083FF23C08091EA
:10432000E100877F8093E10082E080932103109277
:1043300022038091E1008E7F8093E1008091E20072
:104340008E7F8093E2008091E20080618093E200A2
:1043500042E060E080E00E949B248091F000886051
:104360008093F000FF91EF91BF91AF919F918F915A
:104370007F916F915F914F913F912F910F900FBE61
:104380000F901F9018950895809116030895089531
:104390008093AC037093AE036093AD0380912103CF
:1043A000843001F582E08093E9008FEF9091E8007E
:1043B000815095FD06C095ED9A95F1F700008111A9
:1043C000F5CF8091E80085FF0DC040E050E063E04C
:1043D00070E08CEA93E00E942F1D8091E8008E77B8
:1043E0008093E8000895BC0184E00C94C821BC01CE
:1043F00083E00C94C82122E02093E9002FEF309154
:10440000E800215035FD06C035ED3A95F1F7000082
:104410002111F5CF2091E80025FF0BC040E050E0CE
:1044200066E070E00E942F1D8091E8008E778093F7
:10443000E8000895CF93DF9321E02093E9002FEF68
:104440003091E800215035FD06C035ED3A95F1F781
:1044500000002111F5CF2091E80025FF14C0EC01E8
:1044600040E050E068E070E00E942F1D8091E8007D
:104470008E778093E80088E0FE01A7E1B3E0019029
:104480000D928A95E1F7DF91CF910895EF92FF9217
:104490000F931F93CF93DF938C01C1E8D3E0E12CFE
:1044A000F12CF8018481F4E0EF16F1041CF4882368
:1044B00039F002C0811104C09E0140919C0302C0EA
:1044C0009E0140E060919B0380919A030E94D30B70
:1044D0008FEFE81AF80A239698E0E916F10409F735
:1044E0000E94360BF801848190E001968170992733
:1044F0008483DF91CF911F910F91FF90EF900895EA
:104500008F929F92AF92BF92CF92DF92EF92FF92E3
:104510000F931F93CF93DF93EC014C81042F10E096
:104520009801D8010E94B62A9B01AC010E94812A01
:104530006B017C01E0E2F0E0E01BF10BA5E5B0E0EF
:104540009B01AC010E94812A4B015C019F01DF01AC
:104550000E942A2D9B01AC010E948C2A9B01AC0178
:104560002C0D3D1D4E1D5F1DC501B4010E94942AF6
:10457000822FF22E99E2921728F093E0299F900162
:1045800011240DC025E530E0281B3109C901880F31
:10459000991F280F391F37FF02C02F5F3F4F3595F6
:1045A0002795122F109591E8C92E93E0D92E00E09F
:1045B00085E5E82EEF1801FD02C08E2D01C08F2D7C
:1045C0009601412F60919B030E94D30B0F5F83E004
:1045D000C80ED11C083079F70E94360B8C818111EE
:1045E00002C091E003C0803219F49FEF9093D30191
:1045F0009091D301890F8C83DF91CF911F910F91FF
:10460000FF90EF90DF90CF90BF90AF909F908F90F2
:1046100008950F931F93CF93DF93C1E8D3E0FE017A
:10462000118210821282339683E0E939F807C1F7CC
:1046300000E010E080917F03082E000C990B081712
:10464000190794F08091D201082E000C990B801765
:10465000910754F09E0140919C0360919B038091CF
:104660009A030E94D30B03C0198218821A820F5F2B
:104670001F4F239608301105E9F60E94360B8091F2
:10468000D10190917F03980F90937F032091D201E5
:10469000280F2093D201121614F497301CF0819544
:1046A0008093D101DF91CF911F910F910895CF9207
:1046B000DF92EF92FF920F931F93CF93DF93FC0152
:1046C000828180FF03C0DD24DA9402C0DD24D3940C
:1046D000C1E8D3E000E010E0198218821A8294E069
:1046E000E92EF12CC12C80917E038C0D893014F0C1
:1046F000877002C087FD885F082E000C990B081791
:10470000190791F480919C038E9DA0018F9D500DFF
:10471000112455954795559547959E0160919B03AA
:1047200080919A030E94D30BCD0CF1E0EF1AF108AF
:10473000D1F60F5F1F4F23960830110569F60E94CE
:10474000360B80917E0391E0D91206C0811102C020
:1047500087E006C0815004C090E0019687709927D9
:1047600080937E03DF91CF911F910F91FF90EF9087
:10477000DF90CF900895EF92FF921F93CF93DF9336
:10478000EC0181E8E82E83E0F82E10E08C8197019F
:1047900040919C0360919B03810F0E94D30B115E9B
:1047A00083E0E80EF11C183F89F70E94360B9A81CE
:1047B0008C8190FF02C08F5F01C081508C83DF919C
:1047C000CF911F91FF90EF9008950F931F93CF9378
:1047D000DF9300D01F92CDB7DEB78C0180918003AC
:1047E00081110AC09E012F5F3F4F4FEF6FEF0E9474
:1047F000D30B8A8180938003F8018481813051F04A
:1048000028F0823061F4409180030AC080918003D7
:1048100040E007C06091800340E080E003C040E0DA
:1048200080E060E00E946C0BF801848190E00196CA
:1048300063E070E00E94102D84830F900F900F9022
:10484000DF91CF911F910F910895CF93DF93EC01EA
:10485000E9E9F3E0438162818C810E94690C8C81DB
:104860008F5F8C83DF91CF910895CF93DF93EC011D
:10487000EC81F0E0ED5AFC4F4491E9E9F3E062810C
:1048800081810E94690C8C818F5F8C83DF91CF9135
:1048900008952091E4003091E50095E64091EC0008
:1048A000842F817040FF23C08091E80080FD1DC0EF
:1048B00080912103882399F0853099F08091EB0055
:1048C00085FD11C04091E4005091E50024173507A3
:1048D00029F3915011F09A01E1CF84E0089582E02C
:1048E000089583E0089581E0089580E0089540915F
:1048F000E80042FFDDCF08958091230387FF11C0B8
:104900008091E80082FD05C0809121038111F8CFDC
:1049100011C08091E8008B770BC080912103882320
:1049200049F08091E80080FFF8CF8091E8008E7711
:104930008093E8000895982F973068F59093E900E8
:10494000981739F07091EC002091ED005091F00033
:1049500003C0242F762F50E021FD02C09F5FECCFD3
:104960003091EB003E7F3093EB003091ED003D7FC6
:104970003093ED003091EB0031603093EB00709399
:10498000EC002093ED005093F0002091EE0027FD05
:10499000E5CF80E008958F708093E90081E008956D
:1049A0002091290330912A032617370748F0611513
:1049B000710539F42091E8002E772093E80001C0BA
:1049C000B901FC0120E06115710579F180912103A5
:1049D0008823F1F18530F1F18091E80083FD3CC03E
:1049E0008091E80082FD2EC08091E80080FFEBCF2F
:1049F0002091F3008091F20090E0922B61157105F7
:104A000051F08830910538F421912093F1006150E4
:104A100071090196F3CF21E0089709F020E0809119
:104A2000E8008E778093E800CECF2111CFCF0AC067
:104A300080912103882361F0853061F08091E80046
:104A400083FD0AC08091E80082FFF2CF80E00895E4
:104A500082E0089583E0089581E0089581E08093E5
:104A6000E00080E28093D8001092C9008FE19EE4BC
:104A70000197F1F700C0000087E090EBDC01809324
:104A8000B9039093BA03A093BB03B093BC039CE01B
:104A900088E10FB6F894A895809360000FBE9093BC
:104AA0006000FFCF78941F920F920FB60F921124DF
:104AB0008F939F93AF93BF938091A8039091A90385
:104AC000A091AA03B091AB030196A11DB11D8093E3
:104AD000A8039093A903A093AA03B093AB03BF913B
:104AE000AF919F918F910F900FBE0F901F901895CF
:104AF0009C014FB7F8948091A8039091A903A091CD
:104B0000AA03B091AB034FBF821B930B08952FB73D
:104B1000F8948091A8039091A903A091AA03B09161
:104B2000AB032FBF08951F920F920FB60F9211245F
:104B30008F939F93AF93BF938091A703811113C06D
:104B40008091A8039091A903A091AA03B091AB030F
:104B50004196A11DB11D8093A8039093A903A09332
:104B6000AA03B093AB03BF91AF919F918F910F9028
:104B70000FBE0F901F9018959C012A5F3F4FFC01BC
:104B80004281461301C01282019682179307B9F73A
:104B900008959C01FC0132969FEF80E041914617F9
:104BA00089F09F3F19F4411101C0982F8F5F863023
:104BB000A9F79F3F39F0F901E90FF11D97FDFA952B
:104BC0006283089508952091A5033091A6032817C4
:104BD000390771F09093A6038093A503E091A30396
:104BE000F091A403309721F00084F185E02D099421
:104BF00008952091A1033091A2032817390771F07D
:104C00009093A2038093A103E091A303F091A403E6
:104C1000309721F00680F781E02D09940895E09106
:104C2000A303F091A403309721F00190F081E02DCF
:104C3000099480E00895EF92FF920F93CF93DF9352
:104C4000C42FD22FFC0182818823D1F04093A0038E
:104C50000E94872590939F0380939E0380E28C0F90
:104C6000883008F06DC0C77081E001C0880FCA9518
:104C7000EAF7DF91CF910F91FF90EF900C941728F6
:104C80008091A00348134BC080919E0390919F0395
:104C90000E947825883C910508F041C0CD17C9F0E5
:104CA00080E28C0F883040F4C77081E001C0880F2B
:104CB000CA95EAF70E94102880E28D0F883048F4E8
:104CC00081E09D2F977001C0880F9A95EAF70E94A6
:104CD0001728093319F0E12CF12C03C080E5E82EE8
:104CE000F12C802F0E948128E114F10451F08FE90A
:104CF0009FE00197F1F700C0000091E0E91AF10888
:104D0000F3CF802F0E94212880E28D0F8830C0F4DD
:104D1000D77081E001C0880FDA95EAF70AC080E217
:104D20008C0F883068F4C77081E001C0880FCA9585
:104D3000EAF7DF91CF910F91FF90EF900C9410283C
:104D4000DF91CF910F91FF90EF900895909199038B
:104D500090FF04C09695981740F003C0811105C0DC
:104D600090E0961710F40C94A70D61E00C945C0D84
:104D7000882311F0FA0101C0FB01099480E090E062
:104D80000E94F92580E090E00E94E3251092F00255
:104D90000E947B15E9E9F2E086E0DF011D928A9529
:104DA000E9F71092930210929202109294020C94DE
:104DB000B10D8F929F92AF92BF92DF92EF92FF92CE
:104DC0000F931F93CF93DF938090FD029090FE028C
:104DD000A090FF02B09000034091F3025091F402C2
:104DE0006091F5027091F602842A952AA62AB72AC4
:104DF000CFE1D0E025E0929F700111249FE0D92EF1
:104E0000082F10E0D501C4010C2E04C0B695A7955B
:104E1000979587950A94D2F780FD04C0219790F763
:104E200080E014C0DC9EF001DD9EF00D1124EE0D3B
:104E3000FF1DE00FF11FEE0FFF1FE352FE4F8591A4
:104E400094910E945813019749F38C2FDF91CF91D1
:104E50001F910F91FF90EF90DF90BF90AF909F90C8
:104E60008F90089524E0929F900D1124890F682F50
:104E7000669566956695982F977085E0689FB00156
:104E8000112440E050E080E0FB01E40FF51FE15504
:104E9000FC4F208130E0092E02C0369527950A94F8
:104EA000E2F721703327042E01C0220F0A94EAF79B
:104EB000822B4F5F5F4F4530510531F7089524E055
:104EC000929F900D1124890FE82FE695E695E695BF
:104ED000877051E001C0550F8A95EAF785E0E89F99
:104EE000F0011124E155FC4F20E030E070E04081FA
:104EF000CB01022E02C0969587950A94E2F7817045
:104F0000819584278523842781932F5F3F4F253008
:104F1000310569F708956093FD027093FE02809356
:104F2000FF02909300030C94BE260F931F9341E061
:104F300050E060E070E004C0440F551F661F771F0B
:104F40008A95D2F740955095609570958091FD02B5
:104F50009091FE02A091FF02B09100038A019B0193
:104F6000082319232A233B23C901B8011F910F915C
:104F70000C948B270F931F9341E050E060E070E0AA
:104F800004C0440F551F661F771F8A95D2F7809182
:104F9000FD029091FE02A091FF02B09100038A01F0
:104FA0009B01082B192B2A2B3B2BC901B8011F9100
:104FB0000F910C948B276093F3027093F40280930B
:104FC000F5029093F6020C94BE26FC01808191813B
:104FD0000E94671692959F70963079F010F4925067
:104FE00001C09A50923068F4803F69F018F4883E0E
:104FF00040F409C0843F29F406C0883E20F0813F78
:1050000011F080E0089581E008951092F10286E0A9
:10501000E9EAF2E0DF011D928A95E9F70C94BE26D9
:10502000882321F00E9474150C947B150895882321
:1050300039F09091F102892B8093F1020C947B1549
:105040000895882309F45CC0823869F40E940F2611
:1050500081FF56C069E387EA92E00E94C9250E9459
:105060007B1569E30EC0833891F40E940F2680FF00
:1050700047C063E587EA92E00E94C9250E947B153C
:1050800063E587EA92E00E94BC250C947B15843886
:1050900069F40E940F2682FF33C067E487EA92E03A
:1050A0000E94C9250E947B1567E4EBCF9CEF980F07
:1050B000913A10F4682FE5CF90E2980F983050F4B1
:1050C000877091E001C0990F8A95EAF7892F0E94B5
:1050D0007415DBCF9BE5980F933020F480E090E0CF
:1050E0000C94F92598E5980F973120F480E090E032
:1050F0000C94E3258D3E20F00E94DB0D0C94B10D45
:105100000895CF93882309F49EC0C82F8238B1F444
:105110000E940F2681FD97C069E387EA92E00E9412
:10512000C9250E947B152FEF81EE94E0215080402D
:105130009040E1F700C0000069E317C08338E1F454
:105140000E940F2680FD7FC063E587EA92E00E94FF
:10515000C9250E947B152FEF81EE94E021508040FD
:105160009040E1F700C0000063E587EA92E00E940A
:10517000BC25CF910C947B158438B1F40E940F2686
:1051800082FD61C067E487EA92E00E94C9250E941F
:105190007B152FEF81EE94E0215080409040E1F7A5
:1051A00000C0000067E4E1CF8CEF8C0F813A80F4FF
:1051B000E9EAF2E08FEA92E02191C217E1F18E175D
:1051C0009F07D1F76C2F87EA92E00E94C925D1CFC3
:1051D00080E28C0F883068F4C77081E090E001C0F5
:1051E000880FCA95EAF79091F102892B8093F1021A
:1051F000C0CFEBE5EC0FE33040F4F0E0EF5CFD4FA7
:10520000808190E0CF910C94F925E8E5EC0FE7312F
:1052100050F4F0E0EE0FFF1FEC5CFD4F80819181B8
:10522000CF910C94E325CD3E70F08C2F0E94940E0C
:10523000CF910C94B10D6C2F87EA92E00E94BC25AF
:105240000E947B15BFCFCF9108958091B801811145
:1052500022C010927D030E94EF0E1092370310922D
:10526000380310922C0310922B03EDE3F3E080E05F
:1052700090E0A0E8BFEB1182108282839383A48325
:10528000B58317821682389623E0ED37F20799F737
:1052900081E08093B801089562E070E08CEF91E0C6
:1052A0000E94B31C2FEF81EE94E02150804090408B
:1052B000E1F700C000000E94252960913A036E7F4B
:1052C00060933A0387E090E00C942E2A60913A03B1
:1052D000616060933A0387E090E00E942E2A62E0CA
:1052E00070E08CEE91E00C94B31C80913903811135
:1052F00044C080E090E00E94282A893E9E4F11F031
:105300000E94031587E090E00E941A2A80933A03D6
:10531000EDE3F3E080E090E0A0E8BFEB11821082C3
:1053200082839383A483B58317821682389623E001
:10533000ED37F20799F78091390381110CC00E9473
:10534000EF0E259A82E0809380008AE180938100AD
:1053500081E0809339030E94252980913A0380FFE0
:1053600006C063E070E084ED91E00E94B31C0E94EF
:10537000872590932E0380932D0308958F929F92FB
:10538000AF92BF92CF92DF92EF92FF92CF93DF93D3
:10539000EC01688179818A819B81611571058105A4
:1053A000910521F464E279ED8BE597E02DE133EF8F
:1053B00041E050E00E94622A49015A019B01AC0180
:1053C000A7EAB1E40E94812A6B017C01ACEEB4EF44
:1053D000A50194010E948F2ADC01CB018C0D9D1D3B
:1053E000AE1DBF1DB7FF03C00197A109B048888358
:1053F0009983AA83BB839F77DF91CF91FF90EF9032
:10540000DF90CF90BF90AF909F908F9008950E94B3
:10541000BE29089580E091E00E94BE290895A0E091
:10542000B0E08093000190930101A0930201B0933A
:1054300003010895F999FECF92BD81BDF89A99278D
:1054400080B50895A6E1B0E044E050E00C94542A01
:10545000A8E1B0E042E050E00C94542A262FF999DC
:10546000FECF92BD81BDF89A019700B4021639F0C3
:105470001FBA20BD0FB6F894FA9AF99A0FBE089594
:105480000396272F0E942F2A0E942E2A252F0E9442
:105490002F2A242F0C942F2A0196272F0E942F2A7F
:1054A0000C942E2ADC01CB01FC01F999FECF06C039
:1054B000F2BDE1BDF89A319600B40D9241505040D2
:1054C000B8F70895052E97FB1EF400940E94792AE0
:1054D00057FD07D00E94942A07FC03D04EF40C9489
:1054E000792A50954095309521953F4F4F4F5F4F0A
:1054F000089590958095709561957F4F8F4F9F4F40
:1055000008950E94B62AA59F900DB49F900DA49F68
:10551000800D911D11240895B7FF0C94812A0E94DB
:10552000812A821B930B0895A1E21A2EAA1BBB1B92
:10553000FD010DC0AA1FBB1FEE1FFF1FA217B3075F
:10554000E407F50720F0A21BB30BE40BF50B661F75
:10555000771F881F991F1A9469F760957095809539
:1055600090959B01AC01BD01CF010895A29FB001B0
:10557000B39FC001A39F700D811D1124911DB29F87
:10558000700D811D1124911D08955058BB27AA2725
:105590000E94DD2A0C94502C0E94422C38F00E946C
:1055A000492C20F039F49F3F19F426F40C943F2C39
:1055B0000EF4E095E7FB0C94392CE92F0E94612C46
:1055C00058F3BA17620773078407950720F079F438
:1055D000A6F50C94832C0EF4E0950B2EBA2FA02D7B
:1055E0000B01B90190010C01CA01A0011124FF2790
:1055F000591B99F0593F50F4503E68F11A16F0408B
:10560000A22F232F342F4427585FF3CF4695379589
:105610002795A795F0405395C9F77EF41F16BA0B4E
:10562000620B730B840BBAF09150A1F0FF0FBB1FFC
:10563000661F771F881FC2F70EC0BA0F621F731F45
:10564000841F48F4879577956795B795F7959E3FA2
:1056500008F0B0CF9395880F08F09927EE0F979533
:10566000879508950E94152C08F481E008950E9402
:105670004B2B0C94502C0E94492C58F00E94422C29
:1056800040F029F45F3F29F00C94392C51110C940F
:10569000842C0C943F2C0E94612C68F39923B1F365
:1056A000552391F3951B550BBB27AA276217730748
:1056B000840738F09F5F5F4F220F331F441FAA1FDC
:1056C000A9F335D00E2E3AF0E0E832D09150504098
:1056D000E695001CCAF72BD0FE2F29D0660F771F46
:1056E000881FBB1F261737074807AB07B0E809F02C
:1056F000BB0B802DBF01FF2793585F4F3AF09E3FB1
:10570000510578F00C94392C0C94842C5F3FE4F311
:10571000983ED4F3869577956795B795F7959F5FF3
:10572000C9F7880F911D9695879597F90895E1E03F
:10573000660F771F881FBB1F621773078407BA079E
:1057400020F0621B730B840BBA0BEE1F88F7E095F9
:1057500008950E94692C88F09F5798F0B92F9927D7
:10576000B751B0F0E1F0660F771F881F991F1AF04C
:10577000BA95C9F714C0B13091F00E94832CB1E002
:1057800008950C94832C672F782F8827B85F39F001
:10579000B93FCCF3869577956795B395D9F73EF4E5
:1057A00090958095709561957F4F8F4F9F4F08958D
:1057B000E89409C097FB3EF49095809570956195AB
:1057C0007F4F8F4F9F4F9923A9F0F92F96E9BB2761
:1057D0009395F695879577956795B795F111F8CFDD
:1057E000FAF4BB0F11F460FF1BC06F5F7F4F8F4F48
:1057F0009F4F16C0882311F096E911C0772321F03E
:105800009EE8872F762F05C0662371F096E8862FD5
:1058100070E060E02AF09A95660F771F881FDAF72C
:10582000880F9695879597F90895990F0008550F59
:10583000AA0BE0E8FEEF16161706E807F907C0F016
:1058400012161306E407F50798F0621B730B840B1E
:10585000950B39F40A2661F0232B242B252B21F4F8
:1058600008950A2609F4A140A6958FEF811D811D98
:10587000089597F99F6780E870E060E008959FEFD2
:1058800080EC089500240A941616170618060906D7
:10589000089500240A9412161306140605060895A6
:1058A000092E0394000C11F4882352F0BB0F40F42E
:1058B000BF2B11F460FF04C06F5F7F4F8F4F9F4F6E
:1058C000089557FD9058440F551F59F05F3F71F0F0
:1058D0004795880F97FB991F61F09F3F79F0879557
:1058E0000895121613061406551FF2CF4695F1DFE0
:1058F00008C0161617061806991FF1CF8695710570
:10590000610508940895E894BB2766277727CB01A3
:1059100097F908950E94152C08F48FEF08950E94BE
:10592000A22C0C94502C0E94422C38F00E94492C3E
:1059300020F0952311F00C94392C0C943F2C112459
:105940000C94842C0E94612C70F3959FC1F3950FE9
:1059500050E0551F629FF001729FBB27F00DB11DF3
:10596000639FAA27F00DB11DAA1F649F6627B00D83
:10597000A11D661F829F2227B00DA11D621F739F6C
:10598000B00DA11D621F839FA00D611D221F749F7A
:105990003327A00D611D231F849F600D211D822FC1
:1059A000762F6A2F11249F5750409AF0F1F08823E8
:1059B0004AF0EE0FFF1FBB1F661F771F881F915015
:1059C0005040A9F79E3F510580F00C94392C0C945F
:1059D000842C5F3FE4F3983ED4F3869577956795E2
:1059E000B795F795E7959F5FC1F7FE2B880F911D3F
:1059F0009695879597F90895AA1BBB1B51E107C09F
:105A0000AA1FBB1FA617B70710F0A61BB70B881F4E
:105A1000991F5A95A9F780959095BC01CD010895DD
:105A200097FB072E16F4009407D077FD09D00E944B
:105A3000FC2C07FC05D03EF4909581959F4F08956E
:105A4000709561957F4F0895EE0FFF1F0590F491BB
:105A5000E02D09940E94B62A332312F48A1B9B0B73
:105A60000C94342D0E94B62AB7FF0895821B930B25
:105A70000895FC014150504030F001900616D1F7D6
:105A80003197CF010895882799270895FB01DC01FC
:105A900004C08D910190801921F441505040C8F705
:0A5AA000881B990B0895F894FFCFBE
:105AAA0001000000000082420000803F0000DC4349
:105ABA00000040400000DC430000803F0000DC435F
:105ACA0000005C44000080415C978A4400008041E9
:105ADA0052D0A444000080410000DC440000804110
:105AEA0000005C440000004100005C4400000041EA
:105AFA0000005C440000004100005C4400000041DA
:105B0A0048F176440000C04000005C440000C040F8
:105B1A0048F176440000C04000005C440000C040E8
:105B2A0048F176440000C04000005C440000C040D8
:105B3A0048F176440000C04000005C440000C040C8
:105B4A0052D02445000000410000DC44000000411E
:105B5A0052D0A444000040410101191A1B1C1D1E09
:105B6A001F202122C4211A22FB21F721F321C3215C
:105B7A000101020152D0A444000000410000DC44AB
:105B8A000000004152D024450000404100005C441E
:105B9A00000000410000DC44000000410000DC4439
:105BAA000000004100005C440000004100010202C4
:105BBA0002020606060909090909090F0F0F0F0F44
:105BCA000F15151518191919191919191919192348
:105BDA0024818283E200E900EA00B500B600B7003A
:105BEA00CD008301CC008A01920194012102230293
:105BFA0024022502260227022A02B300B4006F00FB
:105C0A0070003233FFF1F090913102020002030278
:105C1A00010200FF0100010000FFFF000001000176
:065C2A00FF0066F567F4BF
:00000001FF
